:1000000000308A00FC2A00000030A1001F08C3391C
:1000100021049F000D30A000A00B0C289F149F18F6
:100020000F281E08A601A500260CA300250CA2007F
:10003000A30CA20CA30CA20CA30CA20C2208AD00D2
:10004000A50DA60DA50DA60DFC30A5050430A1003B
:100050001F08C33921049F000D30A000A00B2E28DB
:100060009F149F1831281E08A801A700280CA30080
:10007000270CA200A30CA20CA30CA20CA30CA20C94
:100080002208AE00270DAB00280DAC00AB0DAC0D67
:10009000FC30AB050C30A1001F08C33921049F00C0
:1000A0000D30A000A00B52289F149F1855281E0841
:1000B000AA01A90000344F308400000803196D28FC
:1000C0000230A100A001A00B6328A10B6228973089
:1000D000A000A00B6928800B60280034CF014F08D6
:1000E000293C031C822805150830A000A00B7628A7
:1000F000000005110330A000A00B7C2800000000C8
:10010000CF0A6F280034CF014F08143C031C9728F6
:1001100005150830A000A00B8B2800000511033046
:10012000A000A00B912800000000CF0A8428003412
:100130000830D002031CA728503084000310800C24
:1001400000080319A728A5280000800BA428003464
:10015000AA08031DB0282908DB3C031CB02885161B
:1001600000340130B800B901BA01BB00BC00CC01B9
:10017000042005118512310BC028BD01BE01C6281F
:10018000B108031DC628BD010130BE002D080F3C7B
:10019000031DCC280E30AD00CE014E08033C031CDD
:1001A000E9280F30AD052D08B4000130B405340B3B
:1001B000E0284E080A3C383E840001308000E528E3
:1001C0004E080A3C383E840080010310AD0CCE0A74
:1001D000CD28851DF8280B30CE004E080E3C031CA0
:1001E000F72838304E0784008001CE0AED281E29FA
:1001F0002E08053C031C0B290B30CE004E080E3C8C
:10020000031C0A2938304E0784000130800085160F
:10021000CE0AFE281E292E08093C03181E290B3081
:10022000CE004E080D3C031C1C2938304E078400BC
:1002300080018516CE0A11290130C6002E08063C21
:10024000031C3C290130C7002E08023C031C2C294A
:10025000C8010130C9003B292E08043C031C342985
:100260000130C800C9013B292E08063C031C3B296C
:100270000130C800C9005729C7012E08083C031CDB
:100280004429C801C90157292E080A3C031C4C29DE
:10029000C8010130C90057292E080C3C031C542901
:1002A0000130C800C90157290130C800C900B30195
:1002B0000330CE004E080F3C031C6D2938304E072A
:1002C00084000310000DB30701304E07383E840050
:1002D0000008B3070230CE075A29490B72290310D0
:1002E000490DB3070330B305B308031D7B29013063
:1002F000CA00CB008F29330B8129CA010130CB0002
:100300008F293308023C031D89290130CA00CB0123
:100310008F293308033C031D8F29CA01CB016E20AE
:1003200083200130CE004E08143C031CAF29383026
:100330004E078400000BA5296E200330CF00C63085
:10034000D0009820CF0B9F29AD2983200330CF0008
:10035000C630D0009820CF0BA829CE0A93290511CA
:10036000A820C830CF005B207D2BA101A201A001F5
:10037000A3015608031DBF2955080319D9291030B8
:10038000D7000310D30DD40DA00DA30D56082302E2
:10039000031DCC2955082002031CD5295508A002AD
:1003A000031CA3035608A3020314A10DA20DD70B2F
:1003B000C1290000032AD201D101D208031DF52969
:1003C0005108123C031CF52905150830A000A00BAC
:1003D000E729000005110330A000A00BED29000063
:1003E0000000D10A0319D20ADD290511D830A00076
:1003F000A00BF82900004F08D4004E08D300D60106
:100400000A30D500B5292208CF002108CE00D2013C
:10041000D10152084F02031C1D2A031D132A4E0846
:10042000510203181D2A0130D00000000000000016
:100430000000D10A0319D20A092A00340420051148
:1004400085122C08CF002B08CE00DB210230CF0014
:10045000CE01DB212608CF002508CE00DB210230AB
:10046000CF00CE01DB210230CF00CE01DB21A8205E
:100470000A30CF005B20812B5008A1014F020318E6
:10048000442A4F08A000502AA0010830D100CF0D07
:10049000A00D500820020318A000A10DD10B472A7F
:1004A000822A0420051185122F0B5D2A0130B00726
:1004B0003008033C031D5D2AAF01310B612AB901ED
:1004C000632A0130B9002E08073C031C6B2ABA01CD
:1004D0000130BB00752A2E080A3C0318732A01302C
:1004E000BA00BB01752ABA01BB01B108031D7D2A00
:1004F0002F0B7D2A0130BA00BB002D08CF0003303E
:10050000D0003C2A2108AD000730AD050430CE00F4
:100510004E08063C031CA02A2D08B4000130B40587
:10052000340B982A38304E078400013080009C2A12
:1005300038304E07840080010310AD0CCE0A882AA3
:10054000310BA82A2F0BA82ABC010130BD00BE0028
:10055000B3010130CE004E08063C031CB62A3830E9
:100560004E0784000008B307CE0AAB2A0130B3055A
:10057000B308031DBD2ABF01BF2A0130BF00CE0151
:100580004E08023C031CC72A6E20CE0AC02A013046
:10059000CF005B200130CE004E08063C031CEB2A46
:1005A00038304E078400000BE12A6E200130CF0066
:1005B0005B200230CF00F830D0009820CF0BDB2A30
:1005C000E92A6E200230CF00F830D0009820CF0BFF
:1005D000E42ACE0ACC2ABF08031DF02A8320F12A80
:1005E0006E200511A8203C30CF005B20310BFB2A88
:1005F0001430CF005B20852B84011F3083051F132F
:1006000083161F149F141F159F15073083129F0018
:10061000703083168F001B30650083121F13831602
:100620001F149F141F119F151F129F161F13831253
:100630009F131F14703083168F00831285120420BD
:100640000130AF00B001851D292B0130B600B70184
:100650002C2BB6010130B7002E080C3C0318382BA8
:10066000B601B7010130B500B1000430B200502B23
:100670002E08033C031C442BB601B7010130B50022
:10068000B1010530B200502B2D080C3C03184C2B47
:10069000B1010330B200502B0130B1000230B20082
:1006A0002D08043C0318562B0420502B2E08043C24
:1006B00003185E2B2E08093C0318602B0420562BD0
:1006C000CD0132084D0203186F2B8516FA30CF008A
:1006D0005B208512FA30CF005B20CD0A612B370BEF
:1006E0007A2B85160230CE00FA30CF005B20CE0B7D
:1006F000742B8512360B7E2BB1287A2B370B822B6D
:0E0700001E2A7E2B350B862B512A822B63007E
:02400E00C43FAD
:00000001FF
